:020000040000FA
:02000000BC2919
:040002000034003492
:08000800F200030EF3000408EE
:10001000F4008312031383130C1DB5290C1122085D
:1000200082071F287F28882890289A28A128AA2894
:10003000B328BB28C028CA28D528DA28E3282308F3
:1000400082072628EC28F128FE280929240882079F
:10005000B5290F2914291B29222927292C293329BD
:100060003A293F2946294E2953295A2963296929C2
:100070006E2975297E2985298A298F2996299F2904
:10008000A629AF298207C034F934A434B034993496
:1000900092348234F8348034903488348334C634D3
:1000A000A13486348E34BF34FE34F7349134AB340B
:1000B000CE34A334C134C7349234AF348934A73436
:1000C0008C34FF349C3487348B34C2348207003440
:1000D0000134013402340334033404340434053469
:1000E00006340634073408340834093409348207E6
:1000F0000F2A142A1C2A322A482A532A602A7422D8
:100100006F2258309500023096000230A200B529C7
:10011000742264309500003096000330A200B529A7
:10012000F4309500013096000430A2003414051A12
:100130003410B529A2013C309500003096008E01A4
:100140001F280830A1003C30950000309600063092
:10015000A200B5298E01A00C0318B5286F22073024
:10016000A2008E01B5297422BB286F2274220830A8
:10017000A2008E01B529A10BAA28A2018E011F2879
:100180000830A1003C309500003096000A30A200F3
:100190008E01B5298E016F2274220310051A0314F3
:1001A000A00C0B30A2008E01B529A10BCA28A20118
:1001B0008E011F2810309500273096006430A5006E
:1001C0000D30A200B529A50BB5293C3095000030B3
:1001D0009600A2018E011F280230A3000930A20060
:1001E000B52983132A308400290884072008800059
:1001F000A90A8E01A80BEE28A30126280430A3002B
:100200008E012A30290784000008A0000530A200D2
:10021000B529A90A8E01A80B0129A30126280130BE
:10022000A2000230A400B529CC30A0000530A20005
:100230000330A400B5294430A0000530A2000430EA
:10024000A400B5290C30A2000530A400B529013066
:10025000A2000630A400B529CC30A0000530A200D1
:100260000730A400B529BE30A0000530A200083038
:10027000A400B5290930A2000930A400B52920083E
:10028000A6000930A2000A30A400B5292008A70062
:10029000A4015830950002309600B5290130A20023
:1002A0000C30A400B5293330A0000530A2000D3079
:1002B000A400B5290130A9000830A8000130A3002E
:1002C0000E30A400B529A4015830950002309600E4
:1002D000B5290130A2001030A400B5295530A00086
:1002E0000530A2001130A400B5290130A900083062
:1002F000A8000330A3001230A400B5294430A000A8
:100300000530A2001330A400B5290C30A20014302F
:10031000A400B5290130A2001530A400B52955303C
:10032000A0000530A2001630A400B5290130A900B4
:100330000830A8000330A3001730A400B529BE3050
:10034000A0000530A2001830A400B5290130A90092
:100350000930A8000130A3001930A400B529A40178
:100360005830950002309600B52974088400730E49
:100370008300F20E720E09000301831203138B0037
:100380008C0083168C008E158312850186018316DE
:1003900001308600303085008117831207309F00BE
:1003A00098019201970183169F0183129001831691
:1003B000811683122030840080010408840A7F3A69
:1003C000031DDC29013090000B3097000C118316BF
:1003D0000C15831258309500023096004C30920074
:1003E0008316633092008C1083120B178B1720300A
:1003F000422083120317A30012304220A2001F30B4
:100400004220A1000C304220A00000008312031300
:100410008C1C082A8C1083120313350877280130AE
:10042000A2000130B500632AA208031D632A01302F
:10043000A4000230B500632AA408031D632A26081D
:10044000B6002708B700B71F2E2AF514B609B7095A
:100450000130B60703080139B7072F2AF51003301A
:10046000B500632A36080F396620BB000310B70CAD
:10047000B60C0310B70CB60C0310B70CB60C031077
:10048000B70CB60CB801B901BA010430B500632A43
:1004900064303602031C502A6430B602B80A632A5C
:1004A0000530B500632A0A303602031C5B2A0A3085
:1004B000B602B90A632A3608BA000630B500632AC4
:1004C0007822B501632A000083120313751C6B2A7E
:1004D00075102223052A7514DA22052A052A051229
:1004E000831605128312080083160516831208006E
:1004F00083172330840083120313F51CA02A1030C5
:1005000042208000840301303902031C932A3908F9
:100510004220800084033A084220800084031F3078
:100520004220800008003A0842207F39800084037E
:100530003B084220800084031F30422080000800D6
:1005400001303802031CB42A38084220800084039A
:1005500039084220800084033A0842208000840346
:100560001F3042208000080001303902031CC92AD4
:1005700039084220800084033A0842207F398000F5
:1005800084033B084220800084031F304220800007
:1005900008003A0842207F39800084033B0842204B
:1005A000800084031F304220800084030C304220EE
:0405B00080000800BF
:0C05B40083120317A408031DE02AE42AA8
:1005C0002408043C0318E62A0430A400A40BEA2AF9
:1005D0000430A4002403203E8400831783120313F5
:1005E000001C8610801C0611001D0613801D86113C
:1005F000001E8612801E8513001F0510801F8613A3
:100600008312031701302402031D0A2B83120313E4
:100610000517080002302402031D122B8312031356
:100620008514080003302402031D1A2B83120313C0
:100630000616080004302402031D212B8312031325
:100640008515080083120313051385100612851102
:10065000861406150617861586168517051486173F
:02066000080090
:02400E00101E82
:00000001FF
